:020000040000FA
:0408000005EF06F00A
:1008100003B20FEF05F0F2B42AEF05F09EB032EF0D
:1008200005F09EB23AEF05F0F2A81AEF04F0F2B22A
:100830001CEF04F0E3EF05F0CD90F2929EA026EFBE
:1008400004F00101463F26EF04F0472B81C185F1FA
:1008500082C186F183C187F184C188F17DC181F1B4
:100860007EC182F17FC183F180C184F179C17DF1C4
:100870007AC17EF17BC17FF17CC180F175C179F1D4
:1008800076C17AF177C17BF178C17CF171C175F1E4
:1008900072C176F173C177F174C178F16DC171F1F4
:1008A0006EC172F16FC173F170C174F169C16DF104
:1008B0006AC16EF16BC16FF16CC170F1CECF69F19D
:1008C000CFCF6AF146C16BF147C16CF1CF6ACE6AF6
:1008D0000101466B476B9E90CD800EBC0E8E0EBA0A
:1008E00075EF04F00E8AE3EF05F00E8C0EBEB1EF4B
:1008F00004F069C16DF16AC16EF16BC16FF16CC139
:1009000070F16DC171F16EC172F16FC173F170C19F
:1009100074F171C175F172C176F173C177F174C16F
:1009200078F175C179F176C17AF177C17BF178C13F
:100930007CF179C17DF17AC17EF17BC17FF17CC10F
:1009400080F17DC181F17EC182F17FC183F180C1DF
:1009500084F181C185F182C186F183C187F184C1AF
:1009600088F10101516B526B536B546B69515127E4
:100970006A5152236B5153236C5154236D515127AB
:100980006E5152236F51532370515423715151278B
:10099000725152237351532374515423755151276B
:1009A000765152237751532378515423795151274B
:1009B0007A5152237B5153237C5154237D5151272B
:1009C0007E5152237F51532380515423815151270B
:1009D00082515223835153238451542385515127EB
:1009E000865152238751532388515423D89054332E
:1009F000533352335133D8905433533352335133EA
:100A0000D890543353335233513369C151F16AC1D1
:100A100052F16BC153F16CC154F1E3EF05F0039255
:100A2000030103EE00F080517F0BE92604C0EFFFC5
:100A3000802B8151805D700BD8A48B820000805187
:100A4000815D700BD8A48B9281518019D8B4079026
:100A5000E3EF05F0F2940101383FE3EF05F0392BA5
:100A6000E3EF05F09E900101463FE3EF05F0472BD1
:100A7000E3EF05F09E92C3CF48F1C4CF49F1C282A3
:100A800007B465EF05F03AC13EF13BC13FF13CC10F
:100A900040F13DC141F151C155F152C156F153C12F
:100AA00057F154C158F1010148514E2749514F2384
:100AB000E86A50230D2E65EF05F04FC14AF150C191
:100AC0004BF14E6B4F6B506B078E0201002FE3EF23
:100AD00005F03C0E006F01015D6776EF05F05E6783
:100AE00076EF05F05F6776EF05F060677AEF05F067
:100AF000AAEF05F061C100F162C101F163C102F129
:100B000064C103F10101010E046F000E056F000EB8
:100B1000066F000E076FE3EC11F000C161F101C137
:100B200062F102C163F103C164F100679FEF05F058
:100B300001679FEF05F002679FEF05F00367AAEFDB
:100B400005F05DC161F15EC162F15FC163F160C139
:100B500064F10E80D57ED5BE34D0D6CF3AF1D7CF52
:100B60003BF138C13CF1E86AE8CF3DF10F8001016B
:100B700047A7C7EF05F00E9A0E9C0E9E0101000ECE
:100B8000516F600E526F3D0E536F080E546F01018E
:100B90003ABFD7EF05F03B67D7EF05F03C67D7EFDB
:100BA00005F03D67D7EF05F0F288DCEF05F0F2982D
:100BB000516B526B536B546BD76AD66A0101386B19
:100BC000396BE3EF05F002C0E0FF005001C0D8FF31
:100BD0001000A6B2E9EF05F00CC0A9FF0BC0A8FFFA
:100BE000A69EA69CA684F29E550EA76EAA0EA76E80
:100BF000A682F28EA694A6B2FBEF05F01200A96EB3
:100C0000A69EA69CA680A8501200076A0E6A0F6ACC
:100C10000F010E0EC16E860EC06E030EC26E0F0166
:100C2000896A110E926E080E8A6EF10E936E8B6AAF
:100C3000800E946EF18E0D6A01014E6B4F6B506BFE
:100C40004A6B4B6B0F01280ED56EF28AB00ECD6E3B
:100C50009D800101516B526B536B546B556B566BFE
:100C6000576B586B596B5A6B5B6B5C6B0E9A0E9C97
:100C70000E9E760ECA6E9D8202013C0E006FCC6AFB
:100C8000160EFFEC05F0E8CF00F1170EFFEC05F0B3
:100C9000E8CF01F1180EFFEC05F0E8CF02F1190ED4
:100CA000FFEC05F0E8CF03F1010103AF72EF06F0AE
:100CB000DAEC12F0160E0C6E00C10BF0E9EC05F048
:100CC000170E0C6E01C10BF0E9EC05F0180E0C6E5E
:100CD00002C10BF0E9EC05F0190E0C6E03C10BF02C
:100CE000E9EC05F000C15DF101C15EF102C15FF107
:100CF00003C160F100C161F101C162F102C163F1A0
:100D000003C164F11A0EFFEC05F0E8CF00F11B0EF1
:100D1000FFEC05F0E8CF01F11C0EFFEC05F0E8CF89
:100D200002F11D0EFFEC05F0E8CF03F1010103AF66
:100D3000C8EF06F0DAEC12F01A0E0C6E00C10BF0E0
:100D4000E9EC05F01B0E0C6E01C10BF0E9EC05F0AF
:100D50001C0E0C6E02C10BF0E9EC05F01D0E0C6EC2
:100D600003C10BF0E9EC05F01A0EFFEC05F0E8CF3B
:100D700000F11B0EFFEC05F0E8CF01F11C0EFFECBB
:100D800005F0E8CF02F11D0EFFEC05F0E8CF03F10E
:100D900000C165F101C166F102C167F103C168F1EB
:100DA000240EAC6E900EAB6E240EAC6E080EB86EB8
:100DB000000EB06E1F0EAF6E0401806B816B0F01D1
:100DC000900EAB6E0F019D8A0301806B816BA26B4D
:100DD0008B9207900001F28EF28C07B0A7EF0FF014
:100DE0000EB0E9EF0AF00301805181197F0BD8B4EE
:100DF000A7EF0FF013EE00F081517F0BE126812B5E
:100E0000E7CFE8FFE00BD8B4A7EF0FF023EE82F0B6
:100E1000A2511F0BD926E7CFDFFFA22BDF50780AA4
:100E2000D8A4A7EF0FF0078061C100F162C101F102
:100E300063C102F164C103F10101040E046F000EED
:100E4000056F000E066F000E076FE3EC11F000AFA8
:100E500033EF07F00101030E616F000E626F000EA9
:100E6000636F000E646F03018251720AD8B4E9EF18
:100E70000AF08251520AD8B4E9EF0AF08251630AAB
:100E8000D8B464EF0CF08251690AD8B4BEEF08F010
:100E900082517A0AD8B4D1EF09F08251490AD8B404
:100EA0005DEF08F08251500AD8B47BEF07F0825111
:100EB000700AD8B4BEEF07F08251540AD8B4E9EFF3
:100EC00007F08251740AD8B42FEF08F099EF0CF0B4
:100ED000040114EE00F080517F0BE12682C4E7FF8D
:100EE000802B12000D0E826F68EC07F00A0E826FE5
:100EF00068EC07F0120083C31EF184C31FF185C3A1
:100F000020F186C321F187C322F188C323F189C36D
:100F100024F18AC325F18BC326F18CC327F101018B
:100F200028EC13F09FEC12F0160E0C6E00C10BF0C3
:100F3000E9EC05F0170E0C6E01C10BF0E9EC05F0C1
:100F4000180E0C6E02C10BF0E9EC05F0190E0C6ED8
:100F500003C10BF0E9EC05F000C15DF101C15EF1E8
:100F600002C15FF103C160F100C161F101C162F131
:100F700002C163F103C164F15DEF08F083C31EF1A8
:100F800084C31FF185C320F186C321F187C322F1F9
:100F900088C323F189C324F18AC325F18BC326F1C9
:100FA0008CC327F1010128EC13F09FEC12F000C173
:100FB0005DF101C15EF102C15FF103C160F100C1E9
:100FC00061F101C162F102C163F103C164F15DEF3E
:100FD00008F083C31EF184C31FF185C320F186C3CB
:100FE00021F187C322F188C323F189C324F18AC385
:100FF00025F18CC326F18DC327F1010128EC13F0F4
:101000009FEC12F00101000E046F000E056F010E3F
:10101000066F000E076FF2EC11F01A0E0C6E00C195
:101020000BF0E9EC05F01B0E0C6E01C10BF0E9ECC6
:1010300005F01C0E0C6E02C10BF0E9EC05F01D0E64
:101040000C6E03C10BF0E9EC05F000C165F101C1C4
:1010500066F102C167F103C168F15DEF08F083C377
:101060001EF184C31FF185C320F186C321F187C31C
:1010700022F188C323F189C324F18AC325F18CC3EB
:1010800026F18DC327F1010128EC13F09FEC12F03B
:101090000101000E046F000E056F010E066F000EB9
:1010A000076FF2EC11F000C165F101C166F102C1F8
:1010B00067F103C168F15DEF08F0160EFFEC05F073
:1010C000E8CF00F1170EFFEC05F0E8CF01F1180EA4
:1010D000FFEC05F0E8CF02F1190EFFEC05F0E8CFC8
:1010E00003F17DEC12F0A9EC10F00401730E826F95
:1010F00068EC07F004012C0E826F68EC07F05DC10C
:1011000000F15EC101F15FC102F160C103F17DEC4C
:1011100012F0A9EC10F00401730E826F68EC07F076
:1011200004012C0E826F68EC07F01A0EFFEC05F03C
:10113000E8CF00F11B0EFFEC05F0E8CF01F11C0E2B
:10114000FFEC05F0E8CF02F11D0EFFEC05F0E8CF53
:1011500003F1B3EC0CF004012C0E826F68EC07F085
:1011600065C100F166C101F167C102F168C103F117
:10117000B3EC0CF072EC07F099EF0CF00401690E7F
:10118000826F68EC07F004012C0E826F68EC07F0A8
:101190000101040E006F000E016F000E026F000EC1
:1011A000036F7DEC12F020C182F40401300E82271F
:1011B00068EC07F021C182F40401300E822768EC4C
:1011C00007F022C182F40401300E822768EC07F098
:1011D00023C182F40401300E822768EC07F024C199
:1011E00082F40401300E822768EC07F025C182F4F6
:1011F0000401300E822768EC07F026C182F4040156
:10120000300E822768EC07F027C182F40401300E0B
:10121000822768EC07F004012C0E826F68EC07F05F
:101220000101030E006F000E016F000E026F000E31
:10123000036F7DEC12F020C182F40401300E82278E
:1012400068EC07F021C182F40401300E822768ECBB
:1012500007F022C182F40401300E822768EC07F007
:1012600023C182F40401300E822768EC07F024C108
:1012700082F40401300E822768EC07F025C182F465
:101280000401300E822768EC07F026C182F40401C5
:10129000300E822768EC07F027C182F40401300E7B
:1012A000822768EC07F004012C0E826F68EC07F0CF
:1012B0000101120E006F000E016F000E026F000E92
:1012C000036F7DEC12F020C182F40401300E8227FE
:1012D00068EC07F021C182F40401300E822768EC2B
:1012E00007F022C182F40401300E822768EC07F077
:1012F00023C182F40401300E822768EC07F024C178
:1013000082F40401300E822768EC07F025C182F4D4
:101310000401300E822768EC07F026C182F4040134
:10132000300E822768EC07F027C182F40401300EEA
:10133000822768EC07F004012C0E826F68EC07F03E
:10134000200EF86EF76AF66A04010900F5CF82F400
:1013500068EC07F00900F5CF82F468EC07F00900AB
:10136000F5CF82F468EC07F00900F5CF82F468EC61
:1013700007F00900F5CF82F468EC07F00900F5CF1B
:1013800082F468EC07F00900F5CF82F468EC07F00E
:101390000900F5CF82F468EC07F072EC07F099EFE2
:1013A0000CF08351630AD8A499EF0CF08451610AC0
:1013B000D8A499EF0CF085516C0AD8A499EF0CF0E1
:1013C0008651410A42E08651440A1BE08651420A96
:1013D000D8B438EF0AF08651350AD8B422EF0EF0AF
:1013E0008651360AD8B477EF0EF08651370AD8B452
:1013F000E0EF0EF08651380AD8B43EEF0FF099EFC7
:101400000CF00798079A04017A0E826F68EC07F0D7
:101410000401780E826F68EC07F00401640E826F9D
:1014200068EC07F081A81CEF0AF00401550E826FEA
:1014300068EC07F021EF0AF004014C0E826F68ECB3
:1014400007F072EC07F099EF0CF00788079A040197
:101450007A0E826F68EC07F00401410E826F68EC2F
:1014600007F00401610E826F68EC07F012EF0AF0DA
:101470000798078A04017A0E826F68EC07F004016E
:10148000420E826F68EC07F00401610E826F68EC17
:1014900007F012EF0AF00101620E046F010E056FF2
:1014A000000E066F000E076F59C100F15AC101F11D
:1014B0005BC102F15CC103F1E3EC11F003BFA8EFE3
:1014C0000AF00E0EFFEC05F0E8CF0CF10F0EFFEC6A
:1014D00005F0E8CF0DF1100EFFEC05F0E8CF0EF1AE
:1014E000110EFFEC05F0E8CF0FF12CEC11F059C113
:1014F00004F15AC105F15BC106F15CC107F1E3ECEF
:1015000011F00782F0EC10F02CEC11F00792F0ECE7
:1015100010F059C100F15AC101F15BC102F15CC187
:1015200003F10792F0EC10F0CC0E046FE00E056FA3
:10153000870E066F050E076FE3EC11F000C10CF18A
:1015400001C10DF102C10EF103C10FF1E0EF0AF08C
:101550000101800E006F1A0E016F060E026F000E61
:10156000036F42C104F143C105F144C106F145C115
:1015700007F1E3EC11F003AFC1EF0AF0DAEC12F07F
:1015800012000E0EFFEC05F0E8CF0CF10F0EFFEC91
:1015900005F0E8CF0DF1100EFFEC05F0E8CF0EF1ED
:1015A000110EFFEC05F0E8CF0FF142C100F143C18D
:1015B00001F144C102F145C103F10782F0EC10F0E2
:1015C0000CC100F10DC101F10EC102F10FC103F117
:1015D00012008251520A03E10E82F0EF0AF00E92DD
:1015E000078455C159F156C15AF157C15BF158C131
:1015F0005CF13EC142F13FC143F140C144F141C100
:1016000045F14AC14CF14BC14DF107940EA027EFB3
:101610000BF00101656714EF0BF0666714EF0BF038
:10162000676714EF0BF0686718EF0BF027EF0BF00C
:101630004BEC0AF065C104F166C105F167C106F122
:1016400068C107F1E3EC11F003BF61EF0CF04BEC64
:101650000AF00101000E046F000E056F010E066F07
:10166000000E076F11EC12F00401720E826F68EC2D
:1016700007F004012C0E826F68EC07F07DEC12F08D
:101680001D6748EF0BF00401200E826F4BEF0BF04B
:1016900004012D0E826F68EC07F024C182F404016E
:1016A000300E822768EC07F025C182F40401300E69
:1016B000822768EC07F004012E0E826F68EC07F0B9
:1016C00026C182F40401300E822768EC07F027C19E
:1016D00082F40401300E822768EC07F004016D0EDD
:1016E000826F68EC07F004012C0E826F68EC07F043
:1016F00042C100F143C101F144C102F145C103F10E
:1017000001017DEC12F0A9EC10F00401480E826F8B
:1017100068EC07F004017A0E826F68EC07F00401B0
:101720002C0E826F68EC07F059C100F15AC101F12B
:101730005BC102F15CC103F101017DEC12F0A9EC87
:1017400010F00401630E826F68EC07F004012C0EA8
:10175000826F68EC07F059C100F15AC101F15BC119
:1017600002F15CC103F101010A0E046F000E056F66
:10177000000E066F000E076FF2EC11F0000E046F02
:10178000120E056F000E066F000E076F11EC12F0BF
:101790007DEC12F01EC182F40401300E822768EC49
:1017A00007F01FC182F40401300E822768EC07F0B5
:1017B00020C182F40401300E822768EC07F021C1B9
:1017C00082F40401300E822768EC07F022C182F413
:1017D0000401300E822768EC07F023C182F4040173
:1017E000300E822768EC07F024C182F40401300E29
:1017F000822768EC07F004012E0E826F68EC07F078
:1018000025C182F40401300E822768EC07F026C15E
:1018100082F40401300E822768EC07F027C182F4BD
:101820000401300E822768EC07F00401730E826F0A
:1018300068EC07F004012C0E826F68EC07F0DAEC1C
:1018400012F04CC100F14DC101F1C2EC0DF00EB22D
:101850002DEF0CF00EA05FEF0CF004012C0E826F48
:1018600068EC07F0200EF86EF76AF66A04010900CA
:10187000F5CF82F468EC07F00900F5CF82F468EC4C
:1018800007F00900F5CF82F468EC07F00900F5CF06
:1018900082F468EC07F00900F5CF82F468EC07F0F9
:1018A0000900F5CF82F468EC07F00900F5CF82F467
:1018B00068EC07F00900F5CF82F468EC07F072ECF1
:1018C00007F00E9099EF0CF00401630E826F68EC44
:1018D00007F004012C0E826F68EC07F09EEC0CF010
:1018E00004012C0E826F68EC07F011EC0DF004017E
:1018F0002C0E826F68EC07F08DEC0DF004012C0EBD
:10190000826F68EC07F00101F80E006FCD0E016FD9
:10191000660E026F030E036FB3EC0CF004012C0E85
:10192000826F68EC07F0A3EC0DF072EC07F099EF12
:101930000CF00301A26B0790A7EF0FF0D8900E0EEA
:10194000FFEC05F0E8CF00F10F0EFFEC05F0E8CF5B
:1019500001F1100EFFEC05F0E8CF02F1110EFFECE3
:1019600005F0E8CF03F10101000E046F000E056FD2
:10197000010E066F000E076F11EC12F07DEC12F0F5
:101980001EC182F40401300E822768EC07F01FC1EB
:1019900082F40401300E822768EC07F020C182F443
:1019A0000401300E822768EC07F021C182F40401A3
:1019B000300E822768EC07F022C182F40401300E59
:1019C000822768EC07F023C182F40401300E8227DD
:1019D00068EC07F024C182F40401300E822768EC21
:1019E00007F025C182F40401300E822768EC07F06D
:1019F00004012E0E826F68EC07F026C182F4040108
:101A0000300E822768EC07F027C182F40401300E03
:101A1000822768EC07F004016D0E826F68EC07F016
:101A20001200120EFFEC05F0E8CF00F1130EFFECF0
:101A300005F0E8CF01F1140EFFEC05F0E8CF02F15C
:101A4000150EFFEC05F0E8CF03F101010A0E046F5B
:101A5000000E056F000E066F000E076FF2EC11F01E
:101A6000000E046F120E056F000E066F000E076F5A
:101A700011EC12F07DEC12F01EC182F40401300E64
:101A8000822768EC07F01FC182F40401300E822720
:101A900068EC07F020C182F40401300E822768EC64
:101AA00007F021C182F40401300E822768EC07F0B0
:101AB00022C182F40401300E822768EC07F023C1B2
:101AC00082F40401300E822768EC07F024C182F40E
:101AD0000401300E822768EC07F004012E0E826F9D
:101AE00068EC07F025C182F40401300E822768EC0F
:101AF00007F026C182F40401300E822768EC07F05B
:101B000027C182F40401300E822768EC07F004013B
:101B1000730E826F68EC07F012000A0EFFEC05F0FE
:101B2000E8CF00F10B0EFFEC05F0E8CF01F10C0E51
:101B3000FFEC05F0E8CF02F10D0EFFEC05F0E8CF69
:101B400003F1C2EF0DF0060EFFEC05F0E8CF00F157
:101B5000070EFFEC05F0E8CF01F1080EFFEC05F0F1
:101B6000E8CF02F1090EFFEC05F0E8CF03F1C2EF78
:101B70000DF00101DAEC12F007844AC100F14BC10B
:101B800001F107940101E80E046F800E056F000E4D
:101B9000066F000E076FF2EC11F0000E046F040EDA
:101BA000056F000E066F000E076F11EC12F0880E25
:101BB000046F130E056F000E066F000E076FE3EC47
:101BC00011F00A0E046F000E056F000E066F000E76
:101BD000076F11EC12F07DEC12F001011D67F6EFBA
:101BE0000DF00401200E826FF9EF0DF004012D0EAF
:101BF000826F68EC07F024C182F40401300E822762
:101C000068EC07F025C182F40401300E822768ECED
:101C100007F026C182F40401300E822768EC07F039
:101C200004012E0E826F68EC07F027C182F40401D4
:101C3000300E822768EC07F00401430E826F68ECD7
:101C400007F0120087C31EF188C31FF189C320F17A
:101C50008AC321F18BC322F18CC323F18DC324F1FC
:101C60008EC325F190C326F191C327F101011D6BAD
:101C700028EC13F09FEC12F00101000E046F000E2F
:101C8000056F010E066F000E076FF2EC11F00E0EDD
:101C90000C6E00C10BF0E9EC05F00F0E0C6E01C1EB
:101CA0000BF0E9EC05F0100E0C6E02C10BF0E9EC44
:101CB00005F0110E0C6E03C10BF0E9EC05F0040108
:101CC0007A0E826F68EC07F004012C0E826F68ECCC
:101CD00007F00401350E826F68EC07F004012C0E4A
:101CE000826F68EC07F09EEC0CF021EF0AF087C3DE
:101CF0001EF188C31FF189C320F18AC321F18BC370
:101D000022F18CC323F18DC324F18EC325F190C33E
:101D100026F191C327F101011D6B28EC13F09FEC14
:101D200012F0880E046F130E056F000E066F000E82
:101D3000076FE7EC11F0000E046F040E056F000E44
:101D4000066F000E076FF2EC11F00101E80E046F50
:101D5000800E056F000E066F000E076F11EC12F07B
:101D60000A0E0C6E00C10BF0E9EC05F00B0E0C6EC8
:101D700001C10BF0E9EC05F00C0E0C6E02C10BF08A
:101D8000E9EC05F00D0E0C6E03C10BF0E9EC05F06B
:101D900004017A0E826F68EC07F004012C0E826F4A
:101DA00068EC07F00401360E826F68EC07F004015E
:101DB0002C0E826F68EC07F08DEC0DF021EF0AF02D
:101DC00087C31EF188C31FF189C320F18AC321F1A3
:101DD0008BC322F18CC323F18DC324F18FC325F172
:101DE00090C326F191C327F1010128EC13F09FEC79
:101DF00012F0000E046F120E056F000E066F000E3B
:101E0000076FF2EC11F001010A0E046F000E056F6E
:101E1000000E066F000E076F11EC12F0120E0C6E22
:101E200000C10BF0E9EC05F0130E0C6E01C10BF0D4
:101E3000E9EC05F0140E0C6E02C10BF0E9EC05F0B4
:101E4000150E0C6E03C10BF0E9EC05F004017A0EDF
:101E5000826F68EC07F004012C0E826F68EC07F0CB
:101E60000401370E826F68EC07F004012C0E826FBC
:101E700068EC07F011EC0DF021EF0AF087C31EF1BA
:101E800088C31FF189C320F18AC321F18BC322F1DA
:101E90008CC323F18DC324F18EC325F190C326F1A9
:101EA00091C327F101011D6B28EC13F09FEC12F098
:101EB000880E046F130E056F000E066F000E076F7D
:101EC000E7EC11F0000E046F040E056F000E066FB4
:101ED000000E076FF2EC11F00101E80E046F800EA6
:101EE000056F000E066F000E076F11EC12F0060E64
:101EF0000C6E00C10BF0E9EC05F0070E0C6E01C191
:101F00000BF0E9EC05F0080E0C6E02C10BF0E9ECE9
:101F100005F0090E0C6E03C10BF0E9EC05F00401AD
:101F20007A0E826F68EC07F004012C0E826F68EC69
:101F300007F00401380E826F68EC07F004012C0EE4
:101F4000826F68EC07F0A3EC0DF021EF0AF081A896
:101F500065EF10F007A81EEF10F00101800E006F72
:101F60001A0E016F060E026F000E036F3EC104F1E0
:101F70003FC105F140C106F141C107F1E3EC11F0A9
:101F800003BF65EF10F0A3EC10F03EC100F13FC1BC
:101F900001F140C102F141C103F10782F0EC10F000
:101FA0000CC104F10DC105F10EC106F10FC107F11D
:101FB000F80E006FCD0E016F660E026F030E036FF9
:101FC000E3EC11F00E0E0C6E00C10BF0E9EC05F025
:101FD0000F0E0C6E01C10BF0E9EC05F0100E0C6E4B
:101FE00002C10BF0E9EC05F0110E0C6E03C10BF011
:101FF000E9EC05F007840101DAEC12F04AC100F1C6
:102000004BC101F107940A0E0C6E00C10BF0E9EC14
:1020100005F00B0E0C6E01C10BF0E9EC05F00C0E97
:102020000C6E02C10BF0E9EC05F00D0E0C6E03C155
:102030000BF0E9EC05F0079865EF10F007AA65EFE3
:1020400010F007840101DAEC12F04AC100F14BC133
:1020500001F10794060E0C6E00C10BF0E9EC05F0DF
:10206000070E0C6E01C10BF0E9EC05F0080E0C6ECA
:1020700002C10BF0E9EC05F0090E0C6E03C10BF088
:10208000E9EC05F0078455C100F156C101F157C1D3
:1020900002F158C103F10794120E0C6E00C10BF04F
:1020A000E9EC05F0130E0C6E01C10BF0E9EC05F044
:1020B000140E0C6E02C10BF0E9EC05F0150E0C6E5F
:1020C00003C10BF0E9EC05F0079A04018051811976
:1020D0007F0B0BE09EA809D014EE00F081517F0B1E
:1020E000E126E750812B0F01AD6EEDEF06F00CC13C
:1020F00000F10DC101F10EC102F10FC103F1000E9B
:10210000046F000E056F010E066F000E076F11ECD5
:1021100012F01DA1A2EF10F01451D8B4A2EF10F0EC
:102120000CC100F10DC101F10EC102F10FC103F1AB
:10213000000E046F000E056F0A0E066F000E076F8B
:1021400011EC12F0120001010C6B0D6B0E6B0F6B9A
:1021500012001EC182F40401300E822768EC07F0E1
:102160001FC182F40401300E822768EC07F020C101
:1021700082F40401300E822768EC07F021C182F45A
:102180000401300E822768EC07F022C182F40401BA
:10219000300E822768EC07F023C182F40401300E70
:1021A000822768EC07F024C182F40401300E8227F4
:1021B00068EC07F025C182F40401300E822768EC38
:1021C00007F026C182F40401300E822768EC07F084
:1021D00027C182F40401300E822768EC07F0120058
:1021E0000101005305E1015303E1025301E1002B1A
:1021F000B3EC11F0DAEC12F02C51006F2D51016F9D
:10220000420E046F4B0E056F000E066F000E076F37
:10221000F2EC11F000C104F101C105F102C106F1B7
:1022200003C107F10CC100F10DC101F10EC102F1B2
:102230000FC103F107B221EF11F0E7EC11F023EF2A
:1022400011F0E3EC11F000C10CF101C10DF102C17C
:102250000EF103C10FF11200DAEC12F04CC100F1E3
:102260004DC101F1060EFFEC05F0E8CF04F1070EB9
:10227000FFEC05F0E8CF05F1080EFFEC05F0E8CF24
:1022800006F1090EFFEC05F0E8CF07F1E3EC11F0E1
:1022900000C118F101C119F102C11AF103C11BF10A
:1022A000290E046F000E056F000E066F000E076FFB
:1022B000F2EC11F0EE0E046F430E056F000E066F88
:1022C000000E076FE7EC11F018C104F119C105F118
:1022D0001AC106F11BC107F1F2EC11F000C110F1B7
:1022E00001C111F102C112F103C113F1120EFFEC91
:1022F00005F0E8CF04F1130EFFEC05F0E8CF05F18F
:10230000140EFFEC05F0E8CF06F1150EFFEC05F01A
:10231000E8CF07F10D0E006F000E016F000E026F87
:10232000000E036FF2EC11F0180E046F000E056F33
:10233000000E066F000E076F11EC12F010C104F1D1
:1023400011C105F112C106F113C107F1E7EC11F05B
:102350006A0E046F2A0E056F000E066F000E076FDF
:10236000E3EC11F01200BF0EFA6E200E2D6F2C6BF5
:10237000D8900037013702370337D8B0C4EF11F0D7
:102380002D2FB9EF11F02C072D070353D8B41200ED
:102390000331070B8009326F03390F0B010F2C6FCC
:1023A00080EC5FF0336F2C0580EC5FF0335D335FC2
:1023B0002C6B3233D8B02C272C3332A9D9EF11F043
:1023C00033512C271200FFEC12F0D8B01200035149
:1023D0000719286FC2EC12F0D8900751031928AFE3
:1023E000800F1200286BE6EC12F0D8A0FCEC12F083
:1023F000D8B01200D1EC12F0DAEC12F01F0E296FF7
:1024000012EC13F00B35D8B0C2EC12F0D8A00335A3
:10241000D8B01200292F00EF12F028B1E9EC12F029
:102420001200286B04510511061107110008D8A0ED
:10243000E6EC12F0D8A0FCEC12F0D8B01200086B59
:10244000096B0A6B0B6B12EC13F01F0E296F12EC69
:1024500013F007510B5DD8A43AEF12F006510A5D54
:10246000D8A43AEF12F00551095DD8A43AEF12F062
:102470000451085DD8A04DEF12F00451085F0551DA
:10248000D8A0053D095F0651D8A0063D0A5F075157
:10249000D8A0073D0B5FD8900081292F27EF12F0BD
:1024A00028B1E9EC12F0286BE6EC12F0D89016ECAB
:1024B00013F007510B5DD8A46AEF12F006510A5DC4
:1024C000D8A46AEF12F00551095DD8A46AEF12F0A2
:1024D0000451085DD8A079EF12F0003F79EF12F0B7
:1024E000013F79EF12F0023F79EF12F0032BD8B4DD
:1024F000120028B1E9EC12F012000101286BE6ECA1
:1025000012F0D8B012001BEC13F0200E296F003728
:1025100001370237033711EE27F00A0E2A6FE7362C
:102520000A0EE75CD8B0E76EE5522A2F8FEF12F063
:10253000292F87EF12F028B11D81D89012000101D8
:102540000A0E286F200E296F11EE1DF028512A6FF8
:102550000A0ED890E652D8B0E726E7322A2FAAEF23
:1025600012F00333023301330033292FA4EF12F0AA
:10257000E750FF0FD8A00335D8B012001DB1E9EC29
:1025800012F01200045100270551D8B0053D012773
:102590000651D8B0063D02270751D8B0073D0327A2
:1025A00012000051086F0151096F02510A6F035167
:1025B0000B6F12000101006B016B026B036B1200C9
:1025C0000101046B056B066B076B12000335D8A085
:1025D00012000351800B001F011F021F031F003F49
:1025E000F9EF12F0013FF9EF12F0023FF9EF12F0AC
:1025F000032B282B032512000735D8A01200075102
:10260000800B041F051F061F071F043F0FEF13F069
:10261000053F0FEF13F0063F0FEF13F0072B282BAA
:10262000072512000037013702370337083709370B
:102630000A370B37120001011D6B1E6B1F6B206BDD
:10264000216B226B236B246B256B266B276B12008F
:102650001E510F0B1E6F1F510F0B1F6F20510F0BC1
:10266000206F21510F0B216F22510F0B226F23512D
:102670000F0B236F24510F0B246F25510F0B256F68
:0E26800026510F0B266F27510F0B276F1200EC
:10BF0000E844F926000C160C2B0C3F0C520C640C68
:10BF1000760C860C960CA50CB30CC10CCF0CDC0C6B
:06BF2000E80CF40C000C1B
:00000001FF
